:100000000C9438000C9453000C9453000C9453003F
:100010000C9453000C9453000C9453000C94530014
:100020000C9453000C9453000C9453000C94530004
:100030000C941E120C9453000C9453000C94530017
:100040000C9453000C944E030C9453000C945300E6
:100050000C940C100C9453000C9453000C9453000B
:100060000C9453000C9453000C9453000C945300C4
:1000700011241FBECFEFD4E0DEBFCDBF11E0A0E062
:10008000B1E0E2E4F7E202C005900D92A438B107B6
:10009000D9F712E0A4E8B1E001C01D92AA38B10777
:1000A000E1F70C9476000C940000CF93DF93CDB76A
:1000B000DEB7E1E3F0E088E08083E4E3F0E08FEF97
:1000C0008083EAE3F0E08EE28083ABE3B0E0EBE331
:1000D000F0E0808182608C93ABE3B0E0EBE3F0E092
:1000E000808180628C93DF91CF910895CF93DF93CD
:1000F000CDB7DEB723970FB6F894DEBF0FBECDBFE6
:100100000E9455000E943B030E943D0E7894A5E397
:10011000B0E0E5E3F0E0808181608C930E941203FF
:100120000E940B060E941F050E948A040E94F4038D
:1001300000C080918601813071F41092860189811E
:100140008F5F89830E94780E19820E94E5120E94B7
:10015000EC110E94FB1180919A01813089F5A5E391
:10016000B0E0E5E3F0E0808184608C930E94490D6B
:1001700080919301882359F40E9468080E949C0989
:100180000E9453070E946B040E94B60612C0809121
:100190000101823034F00E9453070E946B040E94D8
:1001A000B60680910101833024F00E9468080E9405
:1001B0009C09A5E3B0E0E5E3F0E080818B7F8C93C0
:1001C00080918401813071F51092840180919301B6
:1001D000882319F40E94F40306C080910101833042
:1001E00014F00E94F4038091900190919101019686
:1001F0009093910180939001809190019091910151
:100200008D33910569F480918E0190918F01019653
:1002100090938F0180938E01109291011092900122
:100220000E942E0580918501813009F082CF1092C5
:1002300085010E949E1080919301813009F079CF51
:1002400080919201813009F074CF109292018091D7
:100250000101282F332727FD30953B832A838A818C
:100260009B818230910569F02A813B8123303105E1
:10027000A9F08A819B81009709F05BCF0E94DE0381
:1002800058CF0E94E90364E084E00E947A010E9452
:100290000B060E941F050E948A044BCF0E94E903AF
:1002A00064E084E00E947A010E940B060E941F0510
:1002B0000E948A040E94F4033CCFCF93DF93CDB712
:1002C000DEB764E084E00E947A016CE480E00E9482
:1002D0007A0110928601809186018823E1F36AE019
:1002E0008CE60E947A0160E085E00E947A01DF914D
:1002F000CF910895CF93DF93CDB7DEB724970FB694
:10030000F894DEBF0FBECDBF8B836C83ABE3B0E050
:10031000EBE3F0E080818D7F8C9387E08A8340C09F
:10032000ABE3B0E0EBE3F0E08081877F8C930000EB
:100330000000000000008A81282F332727FD309518
:1003400081E090E0022E02C0880F991F0A94E2F724
:10035000982F8B81892389838981882341F0ABE39E
:10036000B0E0EBE3F0E0808184608C9307C0ABE306
:10037000B0E0EBE3F0E080818B7F8C930000000025
:1003800000000000ABE3B0E0EBE3F0E080818860C8
:100390008C9300000000000000008A8181508A8355
:1003A0008A8188230CF0BCCF87E08A8340C0ABE30E
:1003B000B0E0EBE3F0E08081877F8C9300000000E9
:1003C000000000008A81282F332727FD309581E027
:1003D00090E0022E02C0880F991F0A94E2F7982F2E
:1003E0008C81892389838981882341F0ABE3B0E044
:1003F000EBE3F0E0808184608C9307C0ABE3B0E076
:10040000EBE3F0E080818B7F8C9300000000000024
:100410000000ABE3B0E0EBE3F0E0808188608C9318
:1004200000000000000000008A8181508A838A81D8
:1004300088230CF0BCCFABE3B0E0EBE3F0E08081CD
:10044000877F8C93ABE3B0E0EBE3F0E080818B7FC0
:100450008C93ABE3B0E0EBE3F0E0808182608C93BF
:1004600024960FB6F894DEBF0FBECDBFDF91CF91BB
:100470000895CF93DF93CDB7DEB724970FB6F894E6
:10048000DEBF0FBECDBF8C83ABE3B0E0EBE3F0E0AB
:1004900080818D7F8C9387E08A834CC0ABE3B0E092
:1004A000EBE3F0E08081877F8C9300000000000088
:1004B000000000000000000000008A81282F332780
:1004C00027FD309581E090E0022E02C0880F991F31
:1004D0000A94E2F7982F8C8189238B838B811816DD
:1004E00044F4ABE3B0E0EBE3F0E0808184608C9314
:1004F00007C0ABE3B0E0EBE3F0E080818B7F8C934F
:1005000000000000000000000000000000000000EB
:10051000ABE3B0E0EBE3F0E0808188608C93000017
:1005200000000000000000000000000000008A81C0
:1005300081508A838A8188230CF0B0CF1B82ABE381
:10054000B0E0EBE3F0E08081877F8C930000000057
:1005500000000000000000000000000087E08A8327
:100560003DC0ABE3B0E0EBE3F0E0808188608C93CA
:10057000E9E3F0E080818983898199278071907017
:10058000181619068CF48A81282F332727FD3095F9
:1005900081E090E0022E02C0880F991F0A94E2F7D2
:1005A000982F8B81892B8B830000000000000000B6
:1005B0000000000000000000ABE3B0E0EBE3F0E07F
:1005C0008081877F8C930000000000000000000005
:1005D0000000000000008A8181508A838A8188237C
:1005E0000CF0BFCFABE3B0E0EBE3F0E08081877FBE
:1005F0008C93ABE3B0E0EBE3F0E080818B7F8C93F6
:10060000ABE3B0E0EBE3F0E0808182608C938B8120
:10061000992724960FB6F894DEBF0FBECDBFDF91A9
:10062000CF910895CF93DF93CDB7DEB70E945D01E0
:1006300010928401809184018823E1F30E943104A7
:100640000E946E0B10928401809184018823E1F353
:1006500010928401809184018823E1F31092840137
:1006600064E084E00E947A016CE480E00E947A01F8
:10067000DF91CF910895CF93DF93CDB7DEB7E3E558
:10068000F0E082E08083EEE4F0E082E48083E9E55C
:10069000F0E08AE08083DF91CF9108951F920F925E
:1006A0000FB60F9211248F93CF93DF93CDB7DEB7A0
:1006B000809188018F5F80938801809188018834C0
:1006C00059F581E08093870110928801809145025D
:1006D0008F5F8093450280914502843641F41092E9
:1006E000450281E08093840181E0809385018091BF
:1006F0004502823319F481E08093850180914402A0
:100700008F5F80934402809144028A3029F41092D2
:10071000440281E080938601DF91CF918F910F9009
:100720000FBE0F901F901895CF93DF93CDB7DEB714
:1007300062E480E00E947A01109284018091840139
:100740008823E1F3109284016BE689E00E947A012C
:1007500010928601809186018823E1F31092860130
:100760001092460216C080914602682F8AE00E94CD
:100770007A01809146029927FC01E45CFE4F80815A
:10078000682F8BE00E947A01809146028F5F8093F0
:10079000460280914602863330F360EA88E00E9488
:1007A0007A0110928601809186018823E1F36CE43E
:1007B00080E00E947A01DF91CF910895CF93DF937B
:1007C000CDB7DEB762E480E00E947A01DF91CF917D
:1007D0000895CF93DF93CDB7DEB76CE480E00E943D
:1007E0007A01DF91CF910895CF93DF93CDB7DEB734
:1007F00089ED8093460213C060E085E00E947A0193
:1008000080914602682F86E00E947A0164E587E0C5
:100810000E947A01809146028F5F80934602809108
:1008200046028C3D48F385EE8093460213C060E09B
:1008300085E00E947A0180914602682F86E00E943E
:100840007A0164E587E00E947A01809146028F5F19
:100850008093460280914602883E48F3DF91CF9113
:100860000895CF93DF93CDB7DEB764970FB6F894B2
:10087000DEBF0FBECDBF8DE589838EE58A838FE510
:100880008B8389E48C838BE58D838DE18E838CE56E
:100890008F83188680E2898789E28A8786E38B873F
:1008A00081E48C878AE08D8781E48E8783E08F875F
:1008B00086E2888B20E1CE010196AC0162E087E000
:1008C0000E94B50464960FB6F894DEBF0FBECDBF8C
:1008D000DF91CF910895CF93DF93CDB7DEB760E07E
:1008E00085E00E947A016FEC86E00E947A016CE854
:1008F00087E00E947A0161E085E00E947A016BE066
:1009000086E00E947A016DE887E00E947A01DF911B
:10091000CF910895CF93DF93CDB7DEB760E085E048
:100920000E947A0160E286E00E947A0160E887E036
:100930000E947A0160E085E00E947A016EE386E021
:100940000E947A0164E887E00E947A0160E085E015
:100950000E947A016CE586E00E947A0168E887E0EF
:100960000E947A01DF91CF910895CF93DF93CDB7A5
:10097000DEB72D970FB6F894DEBF0FBECDBF8987C7
:100980006A875C874B872D878A85282F33278EE1DE
:1009900090E0A901489F9001499F300D589F300D6C
:1009A000112489859927820F931F98878F838D85BE
:1009B000282F33278F819885820F931F9E838D83E5
:1009C000109246028F8198859C838B8328C08B81EF
:1009D0008A838B819C81892F99278983698185E00E
:1009E0000E947A016A8186E00E947A014091460263
:1009F000842F99279C018B859C85F901E80FF91FAD
:100A00008081982F842F8F5F80934602692F87E023
:100A10000E947A018B819C8101969C838B832B8120
:100A20003C818D819E812817390788F22D960FB65B
:100A3000F894DEBF0FBECDBFDF91CF910895CF9365
:100A4000DF93CDB7DEB78BE091E025E0AC016EE03F
:100A500086E10E94B504DF91CF9108950F931F9313
:100A6000CF93DF93CDB7DEB729970FB6F894DEBFEB
:100A70000FBECDBF1886198620918E0130918F014F
:100A8000CE0102964AE050E0BC01C9010E94491320
:100A9000CE010296DC01FD0101900020E9F73197BB
:100AA000CF018A1B9B0B8983109246021CC0809148
:100AB0004602082F112780914602282F3327CE01A6
:100AC0000296FC01E20FF31F80810E941A06282F74
:100AD000CE010596FC01E00FF11F208380914602B4
:100AE0008F5F8093460280914602282F33278981A9
:100AF000992787FD909528173907CCF280918E01B0
:100B000090918F018A3091058CF4CE01089621E0F6
:100B1000AC016EE086E10E94B504CE01059621E0AD
:100B2000AC016EE087E10E94B50408C0CE010596D5
:100B300022E0AC016EE086E10E94B50420919001B4
:100B400030919101CE0102964AE050E0BC01C9010A
:100B50000E944913CE010296DC01FD0101900020A4
:100B6000E9F73197CF018A1B9B0B898310924602CC
:100B70001CC080914602082F112780914602282F21
:100B80003327CE010296FC01E20FF31F80810E9401
:100B90001A06282FCE010596FC01E00FF11F2083D5
:100BA000809146028F5F8093460280914602282FF3
:100BB00033278981992787FD909528173907CCF22B
:100BC00080919001909191018A3091058CF4CE0131
:100BD000089621E0AC016EE089E10E94B504CE01E7
:100BE000059621E0AC016EE08AE10E94B50408C0E0
:100BF000CE01059622E0AC016EE089E10E94B504C9
:100C000029960FB6F894DEBF0FBECDBFDF91CF910E
:100C10001F910F910895CF93DF93CDB7DEB782E098
:100C200091E029E0AC016EE083E00E94B504DF9121
:100C3000CF910895CF93DF93CDB7DEB722970FB64C
:100C4000F894DEBF0FBECDBF8A838A818D3219F43E
:100C500089E4898309C08A81803319F48AE0898311
:100C600003C08A81805389838981992787FD909564
:100C700022960FB6F894DEBF0FBECDBFDF91CF91A5
:100C800008950F931F93CF93DF93CDB7DEB760978F
:100C90000FB6F894DEBF0FBECDBF85E0FE013C96D7
:100CA000DF01982F1D929A95E9F72091A9013091C3
:100CB000AA01CE0102964AE050E0BC01C9010E949F
:100CC0004913CE010296DC01FD0101900020E9F7F5
:100CD0003197CF018A1B9B0B8983109246021CC05F
:100CE00080914602082F112780914602282F332732
:100CF000CE010296FC01E20FF31F80810E941A06CA
:100D0000282FCE010796FC01E00FF11F2083809170
:100D100046028F5F8093460280914602282F332738
:100D20008981992787FD909528173907CCF2CE0144
:100D30000C9624E0AC016EE080E10E94B5042981AC
:100D4000998183E1382F391BCE010796AC016EE003
:100D5000832F0E94B50460960FB6F894DEBF0FBED5
:100D6000CDBFDF91CF911F910F9108950F931F93E6
:100D7000CF93DF93CDB7DEB765970FB6F894DEBF9C
:100D80000FBECDBFCE010E969A8B898BECE7F1E0BA
:100D9000FC8BEB8BF3E0FD8BEB89FC8900808B896E
:100DA0009C8901969C8B8B8BE989FA8900828989C1
:100DB0009A8901969A8B898B9D8991509D8BED899B
:100DC000EE2351F780915302909154022EE130E0CE
:100DD000B9010E948E13CB019B838A838A819B81F8
:100DE000992314F41B821A82CE0104962A813B8136
:100DF0004AE050E0BC01C9010E944913CE010496AB
:100E0000DC01FD0101900020E9F73197CF018A1B39
:100E10009B0B8983109246021CC080914602082FCA
:100E2000112780914602282F3327CE010496FC011A
:100E3000E20FF31F80810E941A06282FCE01099627
:100E4000FC01E00FF11F2083809146028F5F8093A9
:100E5000460280914602282F33278981992787FDF2
:100E6000909528173907CCF2CE010E9623E0AC01FD
:100E70006EE088E00E94B504298199818BE0382FCB
:100E8000391BCE010996AC016EE0832F0E94B50498
:100E900065960FB6F894DEBF0FBECDBFDF91CF9140
:100EA0001F910F910895CF93DF93CDB7DEB72997A8
:100EB0000FB6F894DEBF0FBECDBF80915B0290915C
:100EC0005C028E5590409C838B838B819C8123E0B8
:100ED00030E0B9010E948E13CB019A838983898106
:100EE0009A818A30910524F089E090E09A83898381
:100EF00089819A81992314F41A82198220918C0194
:100F000030918D0189819A818217930709F4D7C0A6
:100F100089819A81823091052CF460E184E00E94FD
:100F20007A0104C060E084E00E947A0189819A819C
:100F300090938D0180938C0180E88D8384E88E836B
:100F400088E88F8389819A819987888788859985A0
:100F50008430910509F45FC08885998585309105B5
:100F6000DCF4888599858130910509F43FC0888536
:100F70009985823091052CF488859985009779F1BF
:100F800073C08885998582309105B9F188859985E6
:100F900083309105C9F168C08885998587309105AE
:100FA00009F44EC088859985883091055CF4888560
:100FB000998585309105B1F18885998586309105AF
:100FC000C1F152C0888599858830910509F43FC0E8
:100FD000888599858930910509F440C045C080E82D
:100FE0008D8384E88E8388E88F833EC081E88D837B
:100FF00084E88E8388E88F8337C082E88D8384E815
:101000008E8388E88F8330C083E88D8384E88E8365
:1010100088E88F8329C083E88D8385E88E8388E8FC
:101020008F8322C083E88D8386E88E8388E88F8350
:101030001BC083E88D8387E88E8388E88F8314C084
:1010400083E88D8387E88E8389E88F830DC083E8EA
:101050008D8387E88E838AE88F8306C083E88D833B
:1010600087E88E838BE88F8360E085E00E947A01B9
:1010700060E286E00E947A018D81682F87E00E94FD
:101080007A0160E085E00E947A016EE386E00E94CA
:101090007A018E81682F87E00E947A0160E085E006
:1010A0000E947A016CE586E00E947A018F81682FA8
:1010B00087E00E947A0160E084E00E947A0129962C
:1010C0000FB6F894DEBF0FBECDBFDF91CF9108956C
:1010D000CF93DF93CDB7DEB726970FB6F894DEBF78
:1010E0000FBECDBF80914B0290914C0226E130E0C3
:1010F000B9010E948E13CB0106969E838D838D814C
:101100009E8199230CF446C08D819E812AE030E0B7
:10111000B9010E948E13CB018A838D819E812AE0C2
:1011200030E0B9010E948E138983898186958C5F96
:1011300089838A81282F332786E890E0821B930BCE
:101140009C838B8320911201309113018B819C81B0
:101150008217930761F080911201909113010E9410
:1011600021098B819C8169810E945B090AC0909151
:1011700098018981981729F08B819C8169810E944F
:101180005B098981809398018B819C8190931301E5
:10119000809312018D819E8199230CF049C08D812D
:1011A0009E81909581959F4F9E838D838D819E8199
:1011B0002AE030E0B9010E948E13CB018A838D8131
:1011C0009E812AE030E0B9010E948E1389838981D3
:1011D000869589838A8199278A579F4F9C838B8321
:1011E00020911201309113018B819C81821793070A
:1011F00061F080911201909113010E9421098B816D
:101200009C8169810E945B090AC090919801898143
:10121000981729F08B819C8169810E945B098981E3
:10122000809398018B819C8190931301809312018C
:1012300026960FB6F894DEBF0FBECDBFDF91CF91DB
:101240000895CF93DF93CDB7DEB726970FB6F89406
:10125000DEBF0FBECDBF9E838D831C821B821DC04F
:101260008D818A838D819E81892F992789836981C8
:1012700085E00E947A016A8186E00E947A0160E03E
:1012800087E00E947A018D819E814E969E838D8398
:101290008B819C8101969C838B838B819C81883080
:1012A0009105F0F226960FB6F894DEBF0FBECDBFC3
:1012B000DF91CF910895CF93DF93CDB7DEB7279716
:1012C0000FB6F894DEBF0FBECDBF9E838D836F83B4
:1012D0001C821B8223C08D818A838D819E81892FF0
:1012E00099278983698185E00E947A016A8186E075
:1012F0000E947A018F819927FC01EE5CFE4F80816C
:10130000682F87E00E947A018D819E814E969E8390
:101310008D838B819C8101969C838B838B819C81A7
:1013200088309105C0F227960FB6F894DEBF0FBE45
:10133000CDBFDF91CF910895CF93DF93CDB7DEB7C7
:1013400026970FB6F894DEBF0FBECDBF809149023D
:1013500090914A0226E130E0B9010E948E13CB0140
:101360009E838D838D819E8199230CF452C08D8143
:101370009E812AE030E0B9010E948E13CB018A835E
:101380008D819E812AE030E0B9010E948E1389830D
:101390008981869589838A81282F332787E090E089
:1013A000AC01421B530B9A018EE190E0AC01249FEB
:1013B000C001259F900D349F900D11240A969C83A7
:1013C0008B8320911001309111018B819C818217B8
:1013D000930761F080911001909111010E946C0AB5
:1013E0008B819C8169810E94CF0A0AC090919701EC
:1013F0008981981729F08B819C8169810E94CF0A8D
:101400008981809397018B819C81909311018093B6
:1014100010018D819E8199230CF055C08D819E8194
:10142000909581959F4F9E838D838D819E812AE02B
:1014300030E0B9010E948E13CB018A838D819E8199
:101440002AE030E0B9010E948E1389838981869554
:101450008C5F89838A81282F33278EE190E0AC014D
:10146000249FC001259F900D349F900D112486501C
:101470009F4F9C838B8320911001309111018B81B0
:101480009C818217930761F0809110019091110166
:101490000E946C0A8B819C8169810E94CF0A0AC0DC
:1014A000909197018981981729F08B819C8169819E
:1014B0000E94CF0A8981809397018B819C819093B0
:1014C00011018093100126960FB6F894DEBF0FBE6F
:1014D000CDBFDF91CF910895CF93DF93CDB7DEB726
:1014E00026970FB6F894DEBF0FBECDBF9E838D83C7
:1014F0008D819E819C838B8318C08B818A838B8195
:101500009C81892F99278983698185E00E947A01CE
:101510006A8186E00E947A0160E087E00E947A0199
:101520008B819C8101969C838B838D819E819C0104
:10153000275F3F4F8B819C8182179307F0F2809148
:101540009701282F3327C901880F991F820F931FF6
:10155000FC01EA5EFE4F80818823C1F08D819E816F
:1015600082969C838B838B818A838B819C81892F3C
:1015700099278983698185E00E947A016A8186E0E2
:101580000E947A0160E087E00E947A0126960FB6F9
:10159000F894DEBF0FBECDBFDF91CF910895CF93FA
:1015A000DF93CDB7DEB727970FB6F894DEBF0FBE37
:1015B000CDBF9E838D836F838D819E819C838B8322
:1015C00024C08B8189838B819C81892F99278A8371
:1015D0006A8185E00E947A01698186E00E947A0131
:1015E0008F81282F3327C901880F991F820F931FDE
:1015F000FC01EC5EFE4F8081682F87E00E947A013B
:101600008B819C8101969C838B838D819E819C0123
:10161000275F3F4F8B819C818217930790F28D81CA
:101620009E8104969C838B838B8189838B819C8193
:10163000892F99278A836A8185E00E947A016981CE
:1016400086E00E947A018F81282F3327C901880FF5
:10165000991F820F931FFC01EB5EFE4F8081682F64
:1016600087E00E947A018F81282F3327C901880FD4
:10167000991F820F931FFC01EA5EFE4F8081882331
:1016800021F18D819E8182969C838B838B818983BE
:101690008B819C81892F99278A836A8185E00E94AA
:1016A0007A01698186E00E947A018F81282F332791
:1016B000C901880F991F820F931FFC01EA5EFE4F3C
:1016C0008081682F87E00E947A0127960FB6F894F0
:1016D000DEBF0FBECDBFDF91CF910895CF93DF93D3
:1016E000CDB7DEB760E085E00E947A0163E886E06E
:1016F0000E947A0160E987E00E947A0160E085E05B
:101700000E947A0164E886E00E947A0161E987E03C
:101710000E947A0160E085E00E947A0165E886E037
:101720000E947A0162E987E00E947A0160E085E028
:101730000E947A0166E886E00E947A0163E987E008
:101740000E947A0160E085E00E947A0167E886E005
:101750000E947A0164E987E00E947A0160E085E0F6
:101760000E947A0168E886E00E947A0165E987E0D4
:101770000E947A0160E085E00E947A0169E886E0D3
:101780000E947A0166E987E00E947A0160E085E0C4
:101790000E947A016AE886E00E947A0167E987E0A0
:1017A0000E947A0160E085E00E947A0161EA86E0A9
:1017B0000E947A0168E987E00E947A0160E085E092
:1017C0000E947A0162EA86E00E947A0169E987E074
:1017D0000E947A0160E085E00E947A0163EA86E077
:1017E0000E947A016AE987E00E947A0160E085E060
:1017F0000E947A0164EA86E00E947A016BE987E040
:101800000E947A0160E085E00E947A0165EA86E044
:101810000E947A016CE987E00E947A0160E085E02D
:101820000E947A0166EA86E00E947A016DE987E00B
:101830000E947A0160E085E00E947A0167EA86E012
:101840000E947A016EE987E00E947A0160E085E0FB
:101850000E947A0168EA86E00E947A016FE987E0D7
:101860000E947A0160E085E00E947A016FEB86E0D9
:101870000E947A0160EA87E00E947A0160E085E0D8
:101880000E947A0160EC86E00E947A0161EA87E0BA
:101890000E947A0160E085E00E947A0161EC86E0B6
:1018A0000E947A0162EA87E00E947A0160E085E0A6
:1018B0000E947A0162EC86E00E947A0163EA87E086
:1018C0000E947A0160E085E00E947A0163EC86E084
:1018D0000E947A0164EA87E00E947A0160E085E074
:1018E0000E947A0164EC86E00E947A0165EA87E052
:1018F0000E947A0160E085E00E947A0165EC86E052
:101900000E947A0166EA87E00E947A0160E085E041
:101910000E947A0166EC86E00E947A0167EA87E01D
:101920000E947A0160E085E00E947A016DED86E018
:101930000E947A0168EA87E00E947A0160E085E00F
:101940000E947A016EED86E00E947A0169EA87E0E2
:101950000E947A0160E085E00E947A016FED86E0E6
:101960000E947A016AEA87E00E947A0160E085E0DD
:101970000E947A0160EE86E00E947A016BEA87E0BD
:101980000E947A0160E085E00E947A0161EE86E0C3
:101990000E947A016CEA87E00E947A0160E085E0AB
:1019A0000E947A0162EE86E00E947A016DEA87E089
:1019B0000E947A0160E085E00E947A0163EE86E091
:1019C0000E947A016EEA87E00E947A0160E085E079
:1019D0000E947A0164EE86E00E947A016FEA87E055
:1019E0000E947A0160E085E00E947A016BEF86E058
:1019F0000E947A0160EB87E00E947A0160E085E056
:101A00000E947A016CEF86E00E947A0161EB87E028
:101A10000E947A0160E085E00E947A016DEF86E025
:101A20000E947A0162EB87E00E947A0160E085E023
:101A30000E947A016EEF86E00E947A0163EB87E0F4
:101A40000E947A0160E085E00E947A016FEF86E0F3
:101A50000E947A0164EB87E00E947A0161E085E0F0
:101A60000E947A0160E086E00E947A0165EB87E0DF
:101A70000E947A0161E085E00E947A0161E086E0DF
:101A80000E947A0166EB87E00E947A01DF91CF9194
:101A90000895CF93DF93CDB7DEB764970FB6F89470
:101AA000DEBF0FBECDBF83E090E09C8B8B8B1A8294
:101AB000198283E990E09C838B83CFC08B899C89BA
:101AC000FC01E555FE4F80819927CD979A8B898B34
:101AD0008B899C8901969C8B8B8B8B899C89FC01C3
:101AE000E555FE4F80819927CD97988B8F878B89FD
:101AF0009C8901969C8B8B8B8B899C89FC01E5557D
:101B0000FE4F80819927CD979E878D878B899C89F1
:101B100001969C8B8B8B8B899C89FC01E555FE4F34
:101B200080819927CD979C878B878B899C8901968B
:101B30009C8B8B8B89899A899C01220F331F220FE2
:101B4000331F8F8598899595879595958795959558
:101B5000879595958795822B932B9A8789878F8573
:101B600098898F7090709C0122953295307F322732
:101B7000207F32278D859E859595879595958795AC
:101B8000822B932B98878F838D859E858370907091
:101B90009C01002436952795079436952795079440
:101BA000322F202D8B859C85822B932B9E838D83BA
:101BB0008B819C8101979C838B838B819C812FEFF0
:101BC0008F3F920709F44EC089819A819C018091D0
:101BD0007F0190918001F901E80FF91F89858083C9
:101BE00089819A8101969A8389838B819C8101974F
:101BF0009C838B838B819C812FEF8F3F920791F188
:101C000089819A819C0180917F0190918001F901E5
:101C1000E80FF91F8F81808389819A8101969A83C9
:101C200089838B819C8101979C838B838B819C8191
:101C30002FEF8F3F9207B1F089819A819C018091AB
:101C40007F0190918001F901E80FF91F8D81808358
:101C500089819A8101969A8389838B819C810097DF
:101C600009F02CCF10929A0164960FB6F894DEBF5B
:101C70000FBECDBFDF91CF910895CF93DF93CDB746
:101C8000DEB7E9E2F0E082E28083E0E4F0E0108297
:101C9000E0E2F0E082E28083ECE5F0E01082A2E393
:101CA000B0E0E2E3F0E0808181608C93A8E3B0E0F3
:101CB000E8E3F0E0808184608C93EAE2F0E088E978
:101CC0008083E0E4F0E086E88083EBE2F0E082EC01
:101CD0008083E1E2F0E088E98083ECE5F0E086E8EB
:101CE0008083E2E2F0E082EC8083DF91CF9108957F
:101CF000CF93DF93CDB7DEB766970FB6F894DEBF0C
:101D00000FBECDBF1A82198283E289871A8683E6C5
:101D10008B871C861D8685E090E098878F831E82C6
:101D20001D821C821B8215C02B813C81CE0109962D
:101D3000FC01E20FF31F8081282F33278D819E81C4
:101D4000820F931F9E838D838B819C8101969C8340
:101D50008B832B813C818F8198852817390724F349
:101D60008D819E8120E030E1B9010E948E139E8317
:101D70008D838F8198859C8B8B8B8D819E819E8B93
:101D80008D8B8D899E8999232CF48D899E89CF9680
:101D90009E8B8D8B8D899E89082E892F000C881F24
:101DA000990B000C881F991F282F235CCE010996E0
:101DB000EB89FC89E80FF91F20838F8198850196B4
:101DC00098878F83EF81F8858D819E8120E430E0B4
:101DD000B9010E948E13282F235CCE010996E80FCB
:101DE000F91F20838F819885019698878F832F8193
:101DF0003885CE010996FC01E20FF31F8DE0808348
:101E00008F819885019698878F831C821B820FC0D3
:101E10002B813C81CE010996FC01E20FF31F8081EA
:101E20000E94250F8B819C8101969C838B838B81E3
:101E30009C818830910564F366960FB6F894DEBFF6
:101E40000FBECDBFDF91CF910895CF93DF93CDB774
:101E5000DEB721970FB6F894DEBF0FBECDBF8983E2
:101E6000E2E2F0E080819927807290700097C1F3E0
:101E7000E3E2F0E08981808321960FB6F894DEBF1B
:101E80000FBECDBFDF91CF910895CF93DF93CDB734
:101E9000DEB721970FB6F894DEBF0FBECDBF8983A2
:101EA000EBE2F0E080819927807290700097C1F397
:101EB000ECE2F0E08981808321960FB6F894DEBFD2
:101EC0000FBECDBFDF91CF910895CF93DF93CDB7F4
:101ED000DEB726970FB6F894DEBF0FBECDBF9E8348
:101EE0008D838D819E81DC01FD0101900020E9F749
:101EF0003197CF018A1B9B0B9C838B831A8219829B
:101F00000FC029813A818D819E81F901E80FF91F67
:101F100080810E94450F89819A8101969A838983E5
:101F200029813A818B819C818217930750F7809198
:101F300081010E94450F809182010E94450F2696E3
:101F40000FB6F894DEBF0FBECDBFDF91CF910895DD
:101F5000CF93DF93CDB7DEB766970FB6F894DEBFA9
:101F60000FBECDBF9E8B8D8B8D899E894AE050E040
:101F70009E012F5F3F4FB9010E944913CE01019688
:101F80000E94650F66960FB6F894DEBF0FBECDBFF8
:101F9000DF91CF910895CF93DF93CDB7DEB722972E
:101FA0000FB6F894DEBF0FBECDBF8A8387E089836A
:101FB0001FC08A81482F55278981282F332727FD65
:101FC000309581E090E0022E02C0880F991F0A949C
:101FD000E2F7842395231816190624F481E30E945E
:101FE000450F03C080E30E94450F8981815089839A
:101FF00089818823F4F6809181010E94450F8091A8
:1020000082010E94450F22960FB6F894DEBF0FBEE4
:10201000CDBFDF91CF9108951F920F920FB60F920F
:1020200011242F933F938F939F93AF93BF93EF937D
:10203000FF93CF93DF93CDB7DEB72297DEBFCDBF3F
:10204000E3E2F0E0808180938902809189028D3003
:10205000D1F4809199018130B1F4A5E3B0E0E5E3DA
:10206000F0E08081877F8C931092990181E08093CA
:102070009A0180914302992720918902FC01E5553C
:10208000FE4F208348C080919901282F33273A833F
:10209000298389819A81009731F029813A81213001
:1020A000310521F138C080918902833271F4809129
:1020B0009A01882351F481E080939901A5E3B0E06F
:1020C000E5E3F0E0808188608C93109243023091C8
:1020D0004302832F992720918902FC01E555FE4F89
:1020E0002083832F8F5F8093430215C0809143022A
:1020F000992720918902FC01E555FE4F20838091AC
:102100004302863930F4809143028F5F809343020B
:1021100002C0109299012296F894DEBFCDBFDF91E4
:10212000CF91FF91EF91BF91AF919F918F913F918F
:102130002F910F900FBE0F901F901895CF93DF93A4
:10214000CDB7DEB76E970FB6F894DEBF0FBECDBF2A
:102150002091490230914A02CE010B964AE050E0AC
:10216000BC01C9010E94491380E4898384E48A8305
:1021700080E38B831C82CE010B96DC01FD01019074
:102180000020E9F73197CF018A1B9B0B9E01255F49
:102190003F4FAC01B901CE0101960E943913CE0127
:1021A0000196DC01FD0101900020E9F731979F01C4
:1021B0002A1B3B0BCE010196820F931FFC0183E289
:1021C00090E091838083CE0101960E94650F20915B
:1021D0004B0230914C02CE010B964AE050E0BC011C
:1021E000C9010E94491380E4898384E48A8381E3DE
:1021F0008B831C82CE010B96DC01FD010190002037
:10220000E9F73197CF018A1B9B0B9E01255F3F4F5A
:10221000AC01B901CE0101960E943913CE0101969D
:10222000DC01FD0101900020E9F731979F012A1B95
:102230003B0BCE010196820F931FFC0183E290E0DD
:1022400091838083CE0101960E94650F20915302F5
:1022500030915402CE010B964AE050E0BC01C90116
:102260000E94491380E4898388E68A838DE38B8307
:102270001C82CE010B96DC01FD0101900020E9F7E4
:102280003197CF018A1B9B0B9E01255F3F4FAC010D
:10229000B901CE0101960E943913CE010196DC01ED
:1022A000FD0101900020E9F731979F012A1B3B0BAC
:1022B000CE010196820F931FFC0183E290E091838F
:1022C0008083CE0101960E94650F20915B023091C0
:1022D0005C02CE010B964AE050E0BC01C9010E94AD
:1022E000491380E4898386E58A838CE68B831C828C
:1022F000CE010B96DC01FD0101900020E9F731973A
:10230000CF018A1B9B0B9E01255F3F4FAC01B9019A
:10231000CE0101960E943913CE010196DC01FD0128
:1023200001900020E9F731979F012A1B3B0BCE015A
:102330000196820F931FFC0183E290E091838083DA
:10234000CE0101960E94650F20918C0130918D0184
:10235000CE010B964AE050E0BC01C9010E9449132E
:1023600080E4898386E58A8381E48B831C82CE01A5
:102370000B96DC01FD0101900020E9F73197CF01B8
:102380008A1B9B0B9E01255F3F4FAC01B901CE011B
:1023900001960E943913CE010196DC01FD010190E6
:1023A0000020E9F731979F012A1B3B0BCE010196D4
:1023B000820F931FFC0183E290E091838083CE0122
:1023C00001960E94650F6E960FB6F894DEBF0FBEA1
:1023D000CDBFDF91CF910895CF93DF93CDB7DEB717
:1023E000A5E3B0E0E5E3F0E0908182E089278C93FB
:1023F000DF91CF910895CF93DF93CDB7DEB7809172
:102400008B018130C1F480918A01813051F4A5E3C0
:10241000B0E0E5E3F0E080818E7F8C9310928A013A
:102420000AC0A5E3B0E0E5E3F0E0808181608C9331
:1024300081E080938A01DF91CF9108951F920F92DE
:102440000FB60F9211242F933F934F935F936F9387
:102450007F938F939F93AF93BF93EF93FF93CF930C
:10246000DF93CDB7DEB780919B0190919C010097DF
:10247000E9F4E4E4F0E0808191819093A2018093FB
:10248000A101AEE4B0E0EEE4F0E080818F7B8C93BC
:1024900081E090E090939C0180939B01A2E3B0E0E7
:1024A000E2E3F0E0808188608C937CC0E4E4F0E0BB
:1024B000808191819093A00180939F01AEE4B0E070
:1024C000EEE4F0E0808180648C9320919F01309154
:1024D000A0018091A1019091A201A901481B590B73
:1024E000CA0190939E0180939D0110929C011092CD
:1024F0009B01A2E3B0E0E2E3F0E08081877F8C9370
:1025000080919D0190919E018656984090939E01E6
:1025100080939D0180919D0190919E012CE231E07C
:10252000B9010E947A13CB0190939E0180939D0183
:1025300080919D0190919E01992324F410929E0117
:1025400010929D0180919D0190919E01873091058F
:1025500034F086E090E090939E0180939D018091FD
:102560000101282F332727FD309580919D019091FF
:102570009E0128173907B1F080919D0190919E012D
:10258000863091057CF480919D0190919E0180930D
:10259000010181E08093920180919D0190919E01C3
:1025A0000E94A80FDF91CF91FF91EF91BF91AF9162
:1025B0009F918F917F916F915F914F913F912F915B
:1025C0000F900FBE0F901F901895CF93DF93CDB74C
:1025D000DEB780915302909154029093420280930F
:1025E000410220914102309142028091A7019091D5
:1025F000A801A901481B590BCA019093A601809319
:10260000A50180914102909142029093A80180938C
:10261000A7012091A3013091A4018091A50190917F
:10262000A601820F931F9093A4018093A301809130
:1026300094018F5F80939401809194018630B1F46E
:10264000109294018091A3019091A40125E030E0C3
:10265000B9010E948E13CB019093AA018093A90126
:102660001092A4011092A3010E944106DF91CF9124
:102670000895FB01DC010D900020E9F7119741500E
:10268000504028F0019000200D92C9F708951C9247
:102690000895FB019F01E8944230C4F04532B4F440
:1026A0004A3029F497FB1EF4909581959F4F642F33
:1026B00077270E947A13805D8A330CF0895D8193BD
:1026C000CB010097A1F716F45DE251931082C90186
:1026D0000C946A13DC01FC0101900020E9F73297A9
:1026E000AE17BF0730F47C916081708331976D9392
:1026F000F7CF0895AA1BBB1B51E107C0AA1FBB1F40
:10270000A617B70710F0A61BB70B881F991F5A957D
:10271000A9F780959095BC01CD01089597FB092EEE
:1027200007260AD077FD04D0E5DF06D000201AF492
:10273000709561957F4F0895F6F7909581959F4F1D
:022740000895FA
:102742000102125A2C294400000A31000044000000
:102752002300230054646653636552620051610092
:102762005060005060005161005262005363655432
:1027720064666768696A6B6B6A6968675555525522
:102782005552555552555552555552555552555506
:1027920052555552555552555552555552555552F9
:1027A20055555255555255555255555255555255E6
:1027B20055525555555555555555555500000047D7
:0427C200020D0A00FA
:00000001FF
